:020000040000FA
:020000000828CE
:02000800A92A23
:1000100003138312850107309F0083163F3085004C
:100020008601803081000C108312013090000B1784
:100030008B1786011E220C30F421A4017722033095
:10004000A6000230F4210030A0004330A100562267
:10005000C030F4215622A322A1220230F4215622DC
:10006000C030F4215622A322A1220230F4215622CC
:10007000C030F4215622A322A122A60B2128013050
:10008000F421A322962820342034533474346F345E
:100090007034573461340034743463346834203439
:1000A0002F34203420342034003420345434693444
:1000B0006D346534723420347634003465347234EF
:1000C0002E3431342E34303435342034003420345E
:1000D00020346234793420346D342E347934003451
:1000E00061346D3461346D346F3474346F34203462
:1000F00000342034303430342034303430343A3426
:100100003034003430343A34303430342E343034F7
:10011000303420340034820701340234043405348E
:10012000073440344234433445344634A1220C3041
:10013000F4210230F4210030A0007930A1005622D1
:10014000C030F4215622B201B301B401B501B601A9
:10015000AF01051AAE28851ACA28A928A122B00124
:100160000D30F42130088B208038F421051C262125
:10017000851C7721051D8E21851DC321051E96280E
:10018000851EB2283308233C0318C8286522B228EC
:100190000C30F421D1207C2286158519CD288611BA
:1001A00096283C308F00CC308E0083160C148312BE
:1001B0002F1CF128AF01B101AE0C0730A700AE0C27
:1001C000031CED28B10AA70BDF280230A700AD0CF5
:1001D000031CED28B10AA70BE7283108093CB00041
:1001E000F920AF18F528851AD82883160C10831229
:1001F000080030088B208038F421300C0739323E5B
:10020000840030180E29000E0F393038F621B00A5C
:1002100005303002031D0E29C030F42100080F39CB
:100220003038F621B00A840A0A3030020319252931
:1002300002303002203003192329083030022E30DA
:10024000031923293A30F621032908001E309C2285
:100250000518442996309C22851834291E309C228A
:10026000851834294521442902303002031D3E29D6
:100270003308233C03183E2965224429B003300A81
:10028000031D44290930B000080077228615831623
:1002900026309B00831232308400851D64290519A5
:1002A0004D29000883169A001C1555309D00AA3070
:1002B0009D009C149C185A299B0A8312840A37308B
:1002C0000402031D5129742983161C141A089B0A61
:1002D00083128000840A37300402031D6429B001B0
:1002E000F9202030F621B0018611A32208001E302B
:1002F0009C2285188D2996309C2203303002031DE4
:1003000087293308233C0318872965228D29B00AE1
:100310000A303002031D8D29B00108001E309C22D6
:100320000519C22996309C22300C0739323E8400D0
:100330003018B62910308007F0300005A8000230D0
:100340003002031DA5292030AA29301DA9295030CB
:10035000AA2990302802031CB1290319B1290F30B2
:100360008005000E0F393038F621C229800A0F307F
:100370000005093C0318BE29F030800500080F393C
:100380003038F62108001E309C228519F32996305A
:100390009C22300C0739323E84003018E729F030B7
:1003A00000050319D62910308002E22902303002FC
:1003B000031DDC292030E129301DE0295030E129DE
:1003C00090308007000E0F393038F621F3290F30B6
:1003D00000050319ED298003EF2909308007000883
:1003E0000F393038F62108000611F82906150000EB
:1003F0008610FE21250EFE2108220800A5000F30E0
:100400008605F03025058604061400000610080055
:100410008316F03086048312061100008614061439
:1004200006080610A500061406080610A51B0F2ACC
:1004300086108316F03086068312080086100000AE
:100440000611000006100F309C223030FE210530CE
:100450009C223030FE218F223030FE218F2220302E
:10046000FE218F222830F4210830F4210130F421BC
:100470000630F42108008316F03086048312061536
:1004800000008614061406080610F039A500A50E13
:10049000061406080610F039A504A50E861083166A
:1004A000F030860683128F222508080061228A1107
:1004B0000A12A10A0319A00A003E03190800F62136
:1004C000562A20088A0021088200DA30A200AD30C6
:1004D000A3004630842AE730A2001730A30046303C
:1004E000842AED30A2005730A3004630842A6B22C4
:1004F0001E309C22712208000430AC0071221E3094
:100500009C22AC0B7E2A0800241483160C14831240
:100510009C2283160C10831224108611080063306D
:10052000A900922AA90B912A08000A30AA008F225A
:10053000AA0B972A08006430AB009522AB0B9D2ACA
:1005400008000530A42A0A30AC009B22AC0BA52A77
:100550000800F300030E8301F0000A08F1008A018D
:100560000408F200831203130C1CCA2A0C1024186E
:10057000C42A3C308F00CC308E00051ED322051AD1
:100580001623AF1C2F14CA2A22088F0023088E00BE
:10059000083086067208840071088A00700E830095
:1005A000F30E730E0900AE01AD01363084000B234B
:1005B0002E1C0800AE14A0300002031C08002E15EB
:1005C000800184030B232E1C0800AE15603000024E
:1005D000031C08002E16800184030B232E1C080028
:1005E000AE1660300002031C08002E178001840341
:1005F0000B23AE1724300002031C08002D148001C9
:1006000084030B232E1C0800AD14A0300002031C31
:100610000800800108002E10800A00080F390A3CEB
:10062000031D08002E14063080070800AE01AD013E
:100630003630840059232E1C0800AE140008F0390F
:10064000F03C031D0800993080002E1584035923C7
:100650002E1C0800AE150008F039F03C031D080000
:10066000593080002E16840359232E1C0800AE1624
:100670000008F039F03C031D0800593080002E17A7
:10068000840359232E1C0800AE170008F039F03CF3
:10069000031D0800233080002D14840359232E1CD1
:1006A0000800AD140008F039F03C031D0800AF1439
:1006B00008002E10800300080F390F3C031D0800AE
:0806C0002E1406308002080030
:02400E00023F6F
:1042000043006F0070007900720069006700680069
:1042100074002000280043002900200032003000F4
:10422000310030002D003200300031003700200016
:104230006200790020004D002E00590061006D00E1
:1042400061006D006F0074006F00FF00000000004F
:0642500000000000000068
:00000001FF
